:100000005B288F00013007288F00043007289400F8
:1000100010080E02031D0E280F080D0204300318ED
:100020000130031902301405031D013056288C00DD
:100030008417800484138F010D1C8F002520031961
:10004000562825200319562825280C088F0601302C
:100050008D008E0100080C050F06031D08008D0A97
:1000600003198E0F2A28080090018F00FF308F0798
:10007000031C9007031C562803308E00DF304220FB
:1000800036288E01E83E8D008E09FC30031C4B287B
:100090008D07031848288D0700008E0F48280D187B
:1000A00051288D1C55280000552808008313831201
:1000B00003130000080086108316861083120611B1
:1000C00083160611013083128D0005308400013043
:1000D00017200E0896000D08950016081504031D3C
:1000E000942801308D0005308400013017200E085F
:1000F00096000D089500861483168610831206114B
:10010000831606110130831290002C30352006151D
:10011000831606118312861083168610013083120F
:1001200090002C3035206D289D0114309C00A001DA
:1001300014309F0001308D000530840001301720FD
:100140000E0896000D08950001308D0005308400E2
:10015000013017200E0896000D08950016081504AA
:10016000031DDD28861583168611013083128D004C
:1001700005308400013017200E0896000D08950008
:1001800086148316861083120611831606118312B5
:100190008611831686110130831290002C30352091
:1001A00006158316061183128610831686100130F9
:1001B000831290002C303520AE28861183168611CC
:1001C00083129A0101308D00053084000130172020
:1001D0000E0896000D0895001608031D16290A3012
:1001E00015020318162901308D00053084000130F6
:1001F00017200E0896000D089500861483168610A9
:1002000083120615831606110130831290002C30DC
:100210003520061183160611831286108316861068
:100220000130831290002C303520EC281608A200F3
:100230001508A10001308D00053084000130172021
:100240000E0896000D08950022081602031D2C29A1
:100250002108150203192D29DD2801308D000530F4
:100260008400013017200E0896000D089500220822
:100270001602031D3F292108150203194029DD2814
:1002800086158316861183120611831606118312B2
:100290008610831686108312970198010130900012
:1002A000F430352001308518030191000130170228
:1002B00003190130031D0301110503197F290130C2
:1002C0009C020030031C013E9D021D081C04031DFE
:1002D0007F299D0114309C008519712903109D0C04
:1002E0009C0C1B08031D7B2901309B008614831680
:1002F000861083127F299B01861083168610013099
:10030000831205190301910001301802031901300D
:10031000031D030111050319AD2901309F020030AF
:10032000031C013EA00220081F04031DAD29A001EB
:1003300014309F0085199F290310A00C9F0C1E08E4
:10034000031DA92901309E0006158316061183128C
:10035000AD299E01061183160611013083128D000E
:1003600005308400013017200E0896000D08950016
:1003700014302107920022080318013E930016084A
:100380001302031CC929031DD929150812020318D9
:10039000D9291708031DD329861483168610013026
:1003A00083129700D829861083168610831297012E
:1003B0000F2216081504031DDE29A428143021027B
:1003C00092000030031C013E2202930016088E00AA
:1003D00015088D00130890001208042091001608DB
:1003E0008E0015088D0090010301012011050319ED
:1003F000092A1808031D032A061583160611013061
:1004000083129800082A0611831606118312980198
:100410000F2216081504031D0E2AA42852299A013A
:1004200001308D0005308400013017200E08960041
:100430000D0895001430210292000030031C013E8B
:100440002202930016088E0015088D0013089000F4
:10045000120804209100143021079200220803188A
:10046000013E930016088E0015088D0013089000B9
:100470001208012011040319512A01308D000530A2
:100480008400013017200E0896000D08950016080C
:100490001504031D502A01309A00960196309500EC
:1004A0001A2A01301A02031D572A960195010800E5
:1004B00043006F00700079007200690067006800F7
:1004C000740020004C00690063006800740065003F
:1004D0006E00620065007200670065007200200017
:1004E0002D0020005600200031002E003100200099
:1004F000320034002F00310031002F003000340072
:02400E00FB3F76
:00000001FF
